:100000000C945C000C9477010C9479000C947900AA
:100010000C9479000C9479000C9479000C9479007C
:100020000C9479000C9479000C9479000C9479006C
:100030000C9479000C9479000C9479000C9479005C
:100040000C9479000C9479000C9479000C9479004C
:100050000C9479000C9479000C9479000C9479003C
:100060000C9479000C94790009021200010100A09F
:100070001409040000000000000012011001FF003C
:100080000008C016DC0500010102000116034C0047
:100090004500440043006F006E00740072006F0062
:1000A0006C0012036F0062006400650076002E0091
:1000B000610074000403090411241FBECFEFD4E0D3
:1000C000DEBFCDBF11E0A0E0B1E0ECEBF5E002C097
:1000D00005900D92A230B107D9F721E0A2E0B1E07E
:1000E00001C01D92A133B207E1F70E94BD020C943A
:1000F000DC020C940000CF93DF93809117018350B2
:1001000087FD28C0909113019D3211F5883001F5CB
:1001100080911401CCE0D0E0C81BD109C55EDE4F50
:1001200083EC809307018AE580930101109202011C
:100130008881807609F45BC0CE010E948B029F818A
:10014000911104C09E81981708F4892F80930001B3
:10015000109217018091010184FF3CC08091000141
:100160008F3FC1F1C82F893008F0C8E08C1B809305
:1001700000018091070198E8892780930701CC232B
:10018000E1F040911501509116018091020186FF26
:1001900085C0A8E0B1E0FA019C2F84918D9331963F
:1001A0009150D9F72FEF2C0F30E02F5F3F4F240FE6
:1001B000351F30931601209315016C2F88E091E0D4
:1001C0000E947301CC5FCC3019F08FEF8093000157
:1001D000C093010184E199B1947131F48150D9F750
:1001E0001092180110921201DF91CF9108952A8187
:1001F00010921001998191110AC01092110120E111
:1002000031E082E0309316012093150198CF9530AC
:1002100029F42093180120E131E0F4CF963071F5F4
:100220009B81913059F48AE790E090931601809376
:10023000150182E190E49093020181CF923019F48C
:1002400088E690E0F2CF9330A9F7211108C084EB43
:1002500090E0909316018093150184E0EBCF21305C
:1002600019F482EA90E0E1CF223021F78CE890E0A7
:10027000909316018093150186E1DCCF983051F000
:10028000993019F420931A01C6CF81E09A3019F2FF
:1002900080E0C1CF2AE131E081E0B4CFDA01E8E0CB
:1002A000F1E09C2F8D9181939150E1F77BCFE9E6AE
:1002B000F0E0808182608083E89A0895A82FB92FAA
:1002C00080E090E041E050EA609530E009C02D9177
:1002D00082279795879510F084279527305EC8F37D
:1002E0006F5FA8F30895EADF8D939D930895CF93F0
:1002F000CFB7CF93DF93C3954C9BE9F74C9B0BC0D3
:100300004C9B09C04C9B07C04C9B05C04C9B03C039
:100310004C9B01C089C06F93C0911401DD27C55E5D
:10032000DE4F2F9365E54C9B03C02F916F91E6CF75
:100330000F931F934F9320E040E15F9309B1047145
:1003400004FB27F93F9350E03BE039C0147140644F
:100350002F77012F5F5F1EC0406819B114712F778E
:1003600052501FC0406409B12F770471D1F15F5F13
:1003700000C023C0406219B12F77147191F15F5F03
:1003800000C025C004711027515012F45D5F0000B9
:10039000115027952C3F19B1C8F61471012701504F
:1003A00027952C3FC8F64227499309B104711027BD
:1003B0004F73115027952C3FA8F64695469519B1D5
:1003C000147179F00127015027952C3F98F66B5A4C
:1003D00060F3315009B1B0F600C011E01CBB00273A
:1003E00017C03B503195C31BD04011E01CBB0881A6
:1003F000033CF9F00B34E9F0209112011981110F3F
:100400001213EDCF093651F10D3211F0013E39F7DB
:10041000009319013F915F914F911F910F912F917F
:100420006F91CCB3C0FD67CFDF91CF91CFBFCF919C
:10043000189520911901222369F3109117011123B6
:1004400039F534303AF130931701209313011091AC
:1004500014013BE0311B309314011CC000911701C3
:100460000130B4F40AE53091010134FD14C0009369
:100470000101C7E0D1E013C0052710E000C0000073
:100480000BB91AC0052710E0221F1DC010E021C0C3
:100490004AE502C032ED432FC4E1D0E032E01AB1A8
:1004A00014615C9A0BB11AB954E120E865E320FFAE
:1004B00005270BB9279517951C3FF0F66695B8F7F9
:1004C000B1F720FF05270BB9279517951C3FD0F6EC
:1004D0002795179517FF052700001C3F0BB9B0F6AD
:1004E00029913A9519F70B7E10911801110FC651F9
:1004F000D0400BB911F01093120111E01CBB006148
:100500001AB11B7E402F4B7E54E05A95F1F70BB980
:100510001AB94BB97FCFFC018181811114C082814E
:10052000809303018381809304018481809305017A
:1005300085818093060183E091E09093160180937A
:10054000150184E00895813051F49281892F8170E2
:1005500090FF03C0289A80E008952898089582307B
:10056000D1F785B181708093030183E091E090938E
:1005700016018093150181E008959EE088E10FB691
:10058000F894A895809360000FBE909360000E943D
:100590005701549A80E0815039F45498209A789405
:1005A000A8950E947B00FCCFA895EFE9FFE031976A
:0C05B000F1F700C00000EFCFF894FFCF7F
:0205BC00FF5AE4
:00000001FF
